:1000000000308B0010308500003086008316C5302C
:100010008100003085004F30860000309A00831246
:10002000103084008001840A841E1228041E1228C5
:100030008E2111309B229D0012309B22A700A2002E
:1000400013309B22013A031D1B1514309B22013AE9
:10005000031D9B150930A4009B10051262219D20F1
:100060006320A720AF212F284320061F34283D20DE
:100070000310061F080003140800053099004320F0
:10008000990B3F2808001A185428861201089C0072
:100090001C0C7F39031950281E02031C061208008D
:1000A0009E08031D06160800061201089C001C0C81
:1000B0007F3903195F281E02031C861208009E0860
:1000C000031D8616080014089000150891001608F4
:1000D000920017089300940195019601970114303E
:1000E000840075207E208820080008309800061BB8
:1000F00077283420800D980B77280800840A061B87
:100100007F283420800D061B83283420800D0800B2
:10011000840A04309800061B8B283420800C840A43
:10012000061B90283420800C980303199928840317
:100130008B28800E8403800E08000930061B0D3EBC
:100140009900061B9D284320990BA1280800100840
:100150001402031DC12811081502031DC12812082D
:100160001602031DC12813081702031DC128100819
:100170001D02031DC1284320120813020319392947
:10018000C22808009B149708970397030319EC28CB
:100190009703031905109703031985109703031993
:1001A000F2289703031905129703031926219703D1
:1001B000970397030319F728970303190514970367
:1001C0000319851497030319EF28970303190516DC
:1001D00097030319312150291208073C1D291208E1
:1001E000F83E1D291208073C03180D291D29083067
:1001F0009602031C1D290319C12896039603960332
:10020000031905149603031985149603960303191D
:1002100005169603031931215029013E03192621A1
:10022000013E03190512013E013E03198510013EEE
:1002300003190510013E013E5029130803391A061F
:1002400003195029130803399A0050299B1D2F299F
:10025000A80012309B22A700A200280808008511E0
:1002600008009B1D37290130A700A2000800851552
:1002700008001208013A031D4D291B184329FF30BD
:10028000A3000930A4001B18C0211B1850291B14FF
:100290009A0901309A05A52150291B1C50291B10D1
:1002A000432062211208013A03195F2912081F0234
:1002B0000319080012089B22A10098210800A1013F
:1002C0009E0108001A18712986131B1D05151B199C
:1002D0007E219B18080011186F29051008000514CD
:1002E000080005111B1D86171B1986219B18080085
:1002F00011187C29851008008514080002301202AC
:10030000031884290511080005150800023012029F
:1003100003188C29861308008617080010309B22CA
:100320009F009B229E00A10015309B229A0008008E
:1003300010308900120888008E2212089F000800E1
:1003400083168818A12983120800153089001A081D
:1003500088008E2283168818AB29831208009B1010
:1003600021081E020319BF29A20BBF2921081E0262
:10037000031CBC299E03BD299E0A2708A200080071
:10038000A30B0800C4290800FF30A300A40B080039
:10039000F2291B30A50BCD29080005158617A122CF
:1003A00005118613A122CA29DF211208013A031977
:1003B000A728DF211208013A031DD92908009D2032
:1003C000632010081402031DDF2911081502031D04
:1003D000DF2912081602031DDF2913081702031D67
:1003E000DF2908000B30A500C921D421B02201303B
:1003F00028020319132A023028020319202A033085
:10040000280203192E2A043028020319582A05301D
:10041000280203196F2A10080319862A0230A50042
:100420002F30CA21F5290230A500C921D42111306D
:100430008900100888008E220230A500C921F52904
:100440000330A500C921D42112308900B022280828
:1004500088008E220230A500C921F5290430A500AC
:10046000C921D421B0222808013E890010080319AF
:10047000862A0F302802031C422A0230A5002F30A2
:10048000CA21312A2808A500C921D4211008B02288
:100490000310A80DA81F512A0230A5002F30CA2131
:1004A000452A280888008E220230A500C921312A59
:1004B0000530A500C921D421B02203302802031C35
:1004C000662A0230A5002F30CA215B2A133089002A
:1004D000280888008E220230A500C921F52906309F
:1004E000A500C921D421B02203302802031C7D2A93
:1004F0000230A5002F30CA21722A14308900280842
:1005000088008E220230A500C921F529FF30A30002
:100510000830A4000B30A500C921122883168B13C4
:1005200008128811081555308900AA3089008814EE
:100530000811831208008900831608148312080822
:1005400008000B11A6000B1DA32A0B11A60BA32A52
:10055000080028080310A80CA80CA807280A0800FF
:10056000A801901FB62AA80A101FA80A901EBC2A2C
:100570000330A807101EA807901DC22A0930A8073B
:10058000101DA807901C08001B30A807101CA80706
:02059000080061
:02400E00F93F78
:10420000000000001400160019001D002200280004
:104210002F00370040004A00550061006E007C000E
:1042200051002A000100010001000100000000000F
:10423000000000000000000000000000000000007E
:10424000000000000000000000000000000000006E
:10425000000000000000000000000000000000005E
:10426000000000000000000000000000000000004E
:10427000000000000000000000000000000000003E
:00000001FF
